:1000000042C0A3C15BC05AC059C058C057C056C0F7
:1000100055C054C053C052C051C050C04FC04EC054
:100020004DC04CC04BC04AC049C048C047C046C084
:1000300045C044C0090212000101008019090400F2
:1000400000000000000012011001FF000008C016AF
:10005000DC050401010200010E03550053004200BB
:100060006100730070001C037700770077002E009A
:10007000660069007300630068006C002E00640075
:1000800065000403090411241FBECFEFD4E0DEBFD6
:10009000CDBF11E0A0E0B1E0EAE7F1E102C00590D8
:1000A0000D92A230B107D9F721E0A2E0B1E001C082
:1000B0001D92AA34B207E1F72CD85DC8A1CFCF9327
:1000C000DF9360912801635067FD13C08091250183
:1000D000CCE0D0E0C81BD109C45DDE4F8091240183
:1000E0008D3209F44EC08091020187FD98C01092B4
:1000F00028018091010184FF37C0609100016F3FAA
:1001000099F1693008F467C06850609300018091EC
:10011000180198E889278093180168E0809102010E
:1001200087FD15C0E0912601F091270186FF68C088
:10013000A9E1B1E0962F84918D9331969150D9F732
:10014000F0932701E0932601C4E0C60F4FC089E178
:1001500091E08CD6682F893008F4A6C08FEF809389
:100160000001CEE1C093010194E189B1847831F4BA
:100170009150D9F71092290110922301DF91CF916C
:100180000895683009F0B3CF83EC809318018AE5B5
:1001900080930101109202018881807609F049C0A4
:1001A0008A8110922101998191114DC010922201F2
:1001B00021E231E082E030932701209326018F3F36
:1001C000D9F19F81911104C09E81981708F4892F5D
:1001D000809300018CCF109200018091180198E863
:1001E000892780931801611199CFC4E089E191E0DA
:1001F000A8D0CC3009F4B6CF8FEF80930001B2CFF6
:10020000DF01C9E1D1E0962F01C0D9019D012F5F27
:100210003F4FF9018C9189939150B9F791CFCE015D
:10022000A3D68F3FF9F0882309F461CF1092000123
:100230005ECFCE0159D4C3CF988197FD1DC090E801
:1002400090930201C5CF953089F0963009F198302E
:10025000D9F0993099F081E09A3009F080E021E2FC
:1002600031E0A9CF8EE18093010141CF8093290134
:1002700021E231E080E09FCF8E81E1CF80932B019E
:1002800021E231E080E097CF2BE231E081E093CFB3
:100290009B819130F1F09230A1F0933041F080E0F9
:1002A00090E4909302018BCFC4E0C80F9FCF8111DF
:1002B00018C082E890E0909327018093260184E0A3
:1002C000EFCF84E390E0909327018093260182E1B1
:1002D000E7CF86E490E0909327018093260182E1A6
:1002E000DFCF813051F08230D1F688E590E09093F5
:1002F0002701809326018EE0D3CF86E690E090938D
:100300002701809326018CE1CBCFE9E6F0E08081E4
:1003100083608083E89A0895A82FB92F80E090E049
:1003200041E050EA609530E009C02D918227979511
:10033000879510F084279527305EC8F36F5FA8F388
:100340000895EADF8D939D930895CF93CFB7CF9310
:10035000DF93C3954F9BE9F74F9B0BC04F9B09C0A1
:100360004F9B07C04F9B05C04F9B03C04F9B01C0D5
:1003700089C06F93C0912501DD27C45DDE4F2F93A7
:1003800065E54F9B03C02F916F91E6CF0F931F93AD
:100390004F9320E040E15F9309B1047807FB27F910
:1003A0003F9350E03BE039C0147840642F77012F31
:1003B0005F5F1EC0406819B114782F7752501FC07C
:1003C000406409B12F770478D1F15F5F00C023C08A
:1003D000406219B12F77147891F15F5F00C025C09A
:1003E00004781027515012F45D5F000011502795DA
:1003F0002C3F19B1C8F614780127015027952C3FDE
:10040000C8F64227499309B1047810274F73115059
:1004100027952C3FA8F64695469519B1147879F0A2
:100420000127015027952C3F98F66B5A60F3315005
:1004300009B1B0F600C011E01CBB002717C03B504B
:100440003195C31BD04011E01CBB0881033CF9F07F
:100450000B34E9F0209123011981110F1213EDCF14
:10046000093651F10D3211F0013E39F700932A019E
:100470003F915F914F911F910F912F916F91CCB34D
:10048000C0FD67CFDF91CF91CFBFCF91189520915D
:100490002A01222369F310912801112339F5343000
:1004A0003AF13093280120932401109125013BE07B
:1004B000311B309325011CC0009128010130B4F498
:1004C0000AE53091010134FD14C000930101C8E137
:1004D000D1E013C0052710E000C000000BB91AC01E
:1004E000052710E0221F1DC010E021C04AE502C010
:1004F00032ED432FC4E1D0E032E01AB114685F9AC4
:100500000BB11AB954E820E865E320FF05270BB9C1
:10051000279517951C3FF0F66695B8F7B1F720FFC1
:1005200005270BB9279517951C3FD0F627951795EA
:1005300017FF052700001C3F0BB9B0F629913A952B
:1005400019F70B7710912901110FC651D0400BB943
:1005500011F01093230111E01CBB00681AB11B7746
:10056000402F4B7754E05A95F1F70BB91AB94BB9B4
:100570007FCF8EBD0DB407FEFDCF8EB5089521E16E
:1005800096958795779567952A95D1F7209146019D
:100590002617D9F060934601E0914301F0914401A0
:1005A0008DE40995E0914301F091440180E00995C3
:1005B000E0914301F0914401809146010995E09159
:1005C0004301F091440180E0099408958091450130
:1005D0008CBD809142018DBD08958823D1F0883073
:1005E00098F129EB32E030934401209343011092BB
:1005F000420191E0909347018930A9F0C0F08B301F
:1006000021F08C30D1F49093420181E58093450133
:10061000089582E593E090934401809343018CE038
:1006200080934701089582E58093450108958830BD
:1006300021F483E580934501089582E58093450187
:1006400081E080934201089522E533E03093440134
:1006500020934301843049F0A0F4823071F083305C
:1006600041F480E380934701089588E18093470136
:10067000089580EC80934701089580E680934701B8
:1006800008958630B9F358F2873099F783E0809364
:100690004701089526B59091470186B5821B8917B9
:1006A000E0F308951F93CF93DF93182FD8E0C0E0B5
:1006B0000BC02B98110FCC0F1C99CF5F2D9AEADF3E
:1006C0002D98E8DFD15021F017FFF3CF2B9AF2CF0E
:1006D0008C2FDF91CF911F91089584B18C6284B9E2
:1006E0002A982D98D7DF2A9AD5DF2A98809143013E
:1006F00090914401895B924019F01092460108954F
:1007000065DF10924601089584B1837D84B985B177
:10071000837D85B91CBC0895CF93DF93C0E202C0EE
:10072000C15059F1E0914301F09144018CEA0995DF
:10073000E0914301F091440183E50995E091430183
:10074000F091440180E00995D82FE0914301F091A8
:10075000440180E00995D335A1F01CBC9BDF2A9AA7
:1007600099DF2A9897DF8091430190914401895B3A
:100770009240B1F62BDFC150A9F681E0DF91CF9115
:10078000089580E0DF91CF910895CF92DF92EF92AC
:10079000FF926B017C01F3DE8C2D8170880F880F36
:1007A000880FE0914301F091440180620995D701DF
:1007B000C60139E0B695A795979587953A95D1F7F3
:1007C000E0914301F09144010995D701C601B69526
:1007D000A79597958795E0914301F091440109957C
:1007E000E0914301F091440180E0FF90EF90DF90B1
:1007F000CF900994CF92DF92EF92FF920F931F93C5
:10080000CF93DF931F92CDB7DEB76B017C01142F1E
:100810002983B5DE8C2D8170880F880F880FE091B9
:100820004301F091440180640995D701C60159E064
:10083000B695A795979587955A95D1F7E09143017D
:10084000F09144010995D701C601B695A7959795F2
:100850008795E0914301F09144010995E0914301AE
:10086000F0914401812F099529812223A9F01F3796
:1008700089F006B51EE1C701B60187DF8F3761F445
:1008800086B5801B813510F006B511501111F3CFDC
:1008900081E003C08FE0B3D080E00F90DF91CF9173
:1008A0001F910F91FF90EF90DF90CF900895CF921E
:1008B000DF92EF92FF920F931F93CF93DF931F92DC
:1008C000CDB7DEB76B017C01498359DEE09143016E
:1008D000F09144018CE40995D701C60179E0B69501
:1008E000A795979587957A95D1F7E0914301F09177
:1008F00044010995D701C601B695A79597958795A7
:10090000E0914301F09144010995E0914301F09198
:10091000440180E0099549814F3FE1F006B51EE1B1
:10092000C701B60132DF8F3F99F486B5801B813550
:1009300010F006B511501111F3CF81E00F90DF9147
:10094000CF911F910F91FF90EF90DF90CF9008957E
:1009500080E0F4CF8FE053D080E0F0CF1F93CF93AF
:10096000DF931F92CDB7DEB7182FE0914301F091CE
:10097000440180EA99830995E0914301F091440193
:100980009981892F0995E0914301F0914401812FCC
:100990000995E0914301F091440180E00F90DF91CF
:1009A000CF911F9109941F93CF93DF9300D0CDB7C0
:1009B000DEB7182FE0914301F091440180EC6A8387
:1009C00099830995E0914301F09144019981892F20
:1009D0000995E0914301F0914401812F0995E0913F
:1009E0004301F09144016A81862F09958EE107D079
:1009F00080E00F900F90DF91CF911F910895882391
:100A000049F030E026B596B5921B9035E0F33F5F94
:100A10003813F8CF0895259A23982B9A50E217D0CF
:100A20005A95E9F70895AC0188E605D0842F03D0E4
:100A300089E601D0852F0FD028E030E0382780FBF1
:100A4000869506D02A95D1F730FB02D000D0689465
:100A500023982B9A16F02B98239AE0914801F09155
:100A600049013197F0F72D9AE3B1E3FBE09148019A
:100A7000F09149013197F0F72D98089520ECE7DFC8
:100A800046F42A95E1F780E02AE1E5DF2A95E9F7C7
:100A9000DECF28E030E0DBDF869587F938272A951E
:100AA000D1F7D5DF27F9322772F3D1DFD0CFDB01C1
:100AB000742FB9DF84E2BFDFE1DF8D937A95D1F740
:100AC0000895DB01742FAFDF83EFB5DF8DE1B3DF76
:100AD00084E6B1DF8D91AFDF82E7ADDFCFDF8078D5
:100AE000D9F77A9589F70895CF93DF93EC0189813F
:100AF000813089F1823009F4B3C0833009F465C0D4
:100B00008430B1F1873009F486C0853009F411C111
:100B1000863009F4A9C0883009F4E0C0893009F4AE
:100B20000DC18A3009F43CC18B3009F46CC18C30A2
:100B300009F47EC18D3009F490C18E3009F492C160
:100B40008F3009F40CC1803109F431C18F3709F4B9
:100B50004FC180E031C0559A4E9B59C05D9880913D
:100B60000E013BDD10920D015B9AB7DD80E024C0E1
:100B700080910D01811112C04B8150E0542F442708
:100B80008A81482B662757FD6095762F409309018F
:100B900050930A0160930B0170930C018F8190E0D8
:100BA000982F88272E81822B90930801809307012C
:100BB00082E080930F018FEF20E131E03093270135
:100BC00020932601DF91CF910895E0914301F091A8
:100BD00044018A81099580931001E0914301F091CD
:100BE00044018B81099580931101E0914301F091BB
:100BF00044018C81099580931201E0914301F091A9
:100C000044018D8109958093130184E0D5CF5D9ACD
:100C100085E0E3DCA7CF80910D01811112C04B81EB
:100C200050E0542F44278A81482B662757FD609552
:100C3000762F4093090150930A0160930B01709342
:100C40000C018F8190E0982F88272E81822B909322
:100C500008018093070183E080930F018FEFACCFF1
:100C600053DD5B9880E0A8CF80910D01811112C007
:100C70008B8190E0982F88272A81822BAA2797FDC5
:100C8000A095BA2F8093090190930A01A0930B01BC
:100C9000B0930C013C812D81822F8F7080930401D1
:100CA000822F807F40E1849FC0011124830F911D1A
:100CB000909306018093050120FD809303018F81AD
:100CC00090E0982F88272E81822B909308018093A3
:100CD000070181E080930F018FEF6ECF80910D01AE
:100CE000811112C08B8190E0982F88272A81822B56
:100CF000AA2797FDA095BA2F8093090190930A0126
:100D0000A0930B01B0930C01109206011092050103
:100D1000109204018F8190E0982F88272E81822BDA
:100D2000909308018093070184E080930F018FEF77
:100D300043CFF2DC8093100181E03ECF81E08093CD
:100D40000D018A819B81AC81BD81809309019093C3
:100D50000A01A0930B01B0930C0180E02DCF8B8191
:100D600090E0982F88272A81822BAA2797FDA095AB
:100D7000BA2F8093090190930A01A0930B01B093BD
:100D80000C018F8190E0982F88272E81822B9093E1
:100D900008018093070185E080930F018FEF0CCF4E
:100DA0008A8180930E011092100181E005CF8B8122
:100DB00090E0982F88272A81822BAA2797FDA0955B
:100DC000BA2F8093090190930A01A0930B01B0936D
:100DD0000C018F8190E0982F88272E81822B909391
:100DE00008018093070186E080930F018FEFE4CE26
:100DF00081E0809310011092110110921201109263
:100E0000130184E0D9CE8B8190E0982F88272A8126
:100E1000822B90934901809348012A9A229A83E079
:100E2000EEDD2A985B9A80E1EADDF5DD80E0C4CE54
:100E300080EC01DE80E0FFDD8AE0E1DD2A9A85E0DA
:100E4000DEDD2A9885E0DBDD84B1837D84B985B160
:100E5000837D85B95B9880E0AFCE10DE8093100172
:100E600081E0AACE8A81E7DD80E0A6CEEF92FF92F4
:100E70000F931F93CF93DF93E62E50910F012EEF28
:100E8000250F223058F0553009F451C08FEFDF9113
:100E9000CF911F910F91FF90EF9008956623E9F194
:100EA0006091090170910A0140910B0120910C01A0
:100EB000EC01F12C20C0CB0151DD888300910901A8
:100EC00010910A0120910B0130910C010F5F1F4F0F
:100ED0002F4F3F4F0093090110930A0120930B01FC
:100EE00030930C01F3942196FE1461F050910F01A0
:100EF000B801422F232F5230F1F6842F922F45DC78
:100F00008883DCCF87E08F1540F48F2DDF91CF9160
:100F10001F910F91FF90EF90089510920F018E2D69
:100F2000DF91CF911F910F91FF90EF900895462F81
:100F3000BC018091090190910A01B9DD009109017C
:100F400010910A0120910B0130910C010E0D111D21
:100F5000211D311D0093090110930A0120930B01FB
:100F600030930C018E2D93CFDF92EF92FF920F936F
:100F70001F93CF93DF939C01F62E40910F014130D8
:100F800071F0443061F0463009F496C08FEFDF9184
:100F9000CF911F910F91FF90EF90DF900895FF2068
:100FA00009F4B5C05091090170910A0180910B01BB
:100FB00090910C01E901E12CD12C50C02091050148
:100FC00030910601232B09F054C021E04881652FA0
:100FD00011DC209107013091080121503109309333
:100FE000080120930701232BE1F410920F01809157
:100FF000040181FF3BC02091030130E08091050195
:10100000909106012817390789F1609109017091C3
:101010000A0180910B0190910C01488148DCDD248C
:10102000D3940091090110910A0120910B01309194
:101030000C010F5F1F4F2F4F3F4F0093090110937B
:101040000A0120930B0130930C01E3942196EF14D5
:1010500051F140910F01502F712FC901413009F416
:10106000ADCF6881852F972F9EDCB3CFDD24D3943D
:10107000D8CF20E04881652FBDDB809103018150EE
:10108000809303018111A5CF6091090170910A013C
:1010900080910B0190910C01488109DC8091050140
:1010A0008093030196CF8D2DDF91CF911F910F91EA
:1010B000FF90EF90DF900895462FBC0180910901C9
:1010C00090910A01FEDC8091090190910A01A091A2
:1010D0000B01B0910C018F0D911DA11DB11D8093CD
:1010E000090190930A01A0930B01B0930C01809128
:1010F0000701909108018F1991099093080180933D
:101100000701892B21F410920F0181E040CF80E08C
:101110003ECF88E10FB6F894809360001092600093
:101120000FBE579A84B1836084B98AB188628AB944
:10113000289A5E9A109285001092840080E4809331
:10114000800089E08093810081E090E090938900A5
:10115000809388002FEF85EA9EE0215080409040E8
:10116000E1F700C0000083E085BD5798CED87894A1
:0A117000A6D7A5D7FDCFF894FFCF56
:02117A00FF5A1A
:00000001FF
